:020000040000FA
:06000000083002303A282E
:08000800A000030EA100831209
:1000100005191028831601178312B23081002B288E
:1000200083160113831203140B190310A80DA90DD5
:10003000AA0DAB0DAC0DAC16FF302C02031D2B2806
:10004000FA302B02031D2B2831152A08AF0029088E
:10005000AE002808AD008B100B11210E8300A00EFE
:04006000200E090065
:0C007400203084008001840A6030040207
:10008000031C3C281230B00073218316FF2390001C
:10009000831283160C308505870183128501870141
:1000A000073099000030831691009F008312C830FA
:1000B00083168100831231309000003083168C004B
:1000C000831210308B00B92181018E018F010B1139
:1000D0008B100B108C018B177C2031197F2057213E
:1000E000B30B7A28031085190314B90DF0303902C7
:1000F0000319F320BE216C2864003210080031116E
:100100000130B7008B132030370783169B001C1477
:100110001A088312A4001030370783169B001C14A2
:100120001A088312A300A6000230A6060030370783
:1001300083169B001C141A088312A200A70001302A
:10014000A7068B17321CAA2822090339A200A3098B
:10015000A409A50924082F02031DED2823082E0257
:10016000031DC92822082D02031DED280130370286
:10017000031DC028BF283D18C0283D143E148F2100
:1001800002303702031DC928BD18C928BD143E140A
:10019000972126082E02031DE52827082D02031D9E
:1001A000ED2801303702031DDB28DA283D1CDB284F
:1001B0003D103E149A2102303702031DE428BD1C75
:1001C000E428BD103E14A221ED285F08AB3C0319C2
:1001D000ED282E1AED28EC28A521B70A03303702A6
:1001E0000318080082280130B600B300B400B5003F
:1001F000B70085018701B113B2217C20B30B2529FB
:10020000031085190314B90DF030390203194C2974
:10021000B41F8501B41F8701B40B252902303702B2
:1002200003191629B50B25290230B5000130370214
:100230000319A821023037020319AD21FA30B400A6
:100240000230370296300319B400311DFD283111F8
:10025000321C2F292D090339AD00AE09AF092F1C1F
:10026000FD288E018F010C1CFD280C102E1EFD2870
:100270008B1320303707BB002F08BA0060211030E5
:100280003707BB002E08BA00602100303707BB00DB
:100290002D08BA0060218B17B52185018701B70AA7
:1002A000B60103303702031CFD28B92108003E1CAB
:1002B00008003E101030BB003D08BA006021080065
:1002C0008B133A0883161C159A003B089B00553087
:1002D0009D00AA309D009C1464009C186C291C1180
:1002E00083128B170800831600309B001C141A0819
:1002F0008312DF00831610309B001C141A0883122F
:10030000BD00831620309B001C141A088312C10004
:100310000130C11BC100C1080319C100080005124A
:1003200005148E018F010C104108C00008008512D1
:1003300085140800051005168E018F010C10410868
:10034000C000080085168510080005100512080079
:10035000380911398500B8000800380922398500AC
:10036000B8000800B80138140800B801B814B8166D
:100370000800BD188514BD1C851608000C1C6C28CF
:100380000C10C00B6C284108C000051005120800B5
:084000000A00030005000100A5
:02400E00CC01E3
:10420000010078007A007C007E007B0079007F004E
:104210007D007A0078007E007C00FF00FF00FF0038
:104220000000F200F600FA00FE00F200F600FA00CC
:10423000FE00F200F600FA00FE00FF00FF00FF00A3
:10424000010005000500050005000900090009003E
:1042500009000D000D000D000D00FF00FF00FF0024
:10426000FF00FF00FF00FF00FF00FF00FF00FF0056
:10427000FF00FF00FF00FF00FF00FF00FF00FF0046
:10428000FF00FF00FF00FF00FF00FF00FF00FF0036
:10429000FF00FF00FF00FF00FF00FF00FF00FF0026
:1042A000FF00FF00FF00FF00FF00FF00FF00FF0016
:1042B000FF00FF00FF00FF00FF00FF00FF00FF0006
:1042C000FF00FF00FF00FF00FF00FF00FF00FF00F6
:1042D000FF00FF00FF00FF00FF00FF00FF00FF00E6
:1042E000FF00FF00FF00FF00FF00FF00FF00FF00D6
:1042F000FF00FF00FF00FF00FF00FF00FF00DD00E8
:00000001FF
